:02000000040AF0
:080008009F0C0200080C060029
:10001000740A000000000000110C27000000E70235
:100020000E0A00084B0C2800F90C29000000E90218
:10003000160AE802140A000866061C0A09090909DA
:1000400066061C0A6607220A09090909090909093D
:1000500009090909090909090909090966071C0AA1
:10006000090909090909090909096607770A090936
:100070000909090909096607840A090909096607BE
:10008000000809090909090909096607840A770AA4
:100090006606480A090909096606480A66074E0AFB
:1000A00009090909090909090909090909090909C0
:1000B000090909096607480A090909090909090915
:1000C00009096607770A090909090909090966077B
:1000D000840A090909096607870A0909090909093A
:1000E00009096607840A770A070C2600480A060CE5
:1000F00026001209000C26001209060C260012091F
:10010000000C26001209480A060C2600480A070CB3
:10011000260012091C09060C260012091C09070CEE
:10012000260012091C09060C260012091C09070CDE
:10013000260012091C09060C260012091C09070CCE
:10014000260012091C09070C260012091C09070CBD
:10015000260012091C09070C260012091C09070CAD
:10016000260012091C09070C260012091C09070C9D
:10017000260012091C0912091C0912091C0912097E
:100180001C0912091C0912091C0912091C0912096F
:100190001C0912091C0912091C0912091C0912095F
:1001A0001C0912091C0912091C0912091C0912094F
:1001B0001C09050C26001209000C26001209050C6A
:1001C00026001209000C2600120912091209120950
:1001D0001C09030C26001209000C26001209030C4E
:1001E00026001209000C2600120912091209120930
:0401F0001C09D90A03
:021FFE00E90FE9
:00000001FF
